:100000000C94A3000C94CB000C94CB000C94CB006C
:100010000C94CB000C94CB000C94CB000C94CB0034
:100020000C94CB000C94CB000C94CB000C94CB0024
:100030000C94CB000C94CB000C94CB000C94CB0014
:100040000C94B4020C94CB000C94CB000C94CB0019
:100050000C94CB000C94CB000C94CB000C94CB00F4
:100060000C94CB000C94CB0007634236B79BD8A707
:100070001A39685618AEBAAB558C1D3CB7CC5763CD
:10008000BD6DEDFD753EF6177231BF000000803F7B
:1000900008000000BE922449123EABAAAA2ABECD97
:1000A000CCCC4C3E00000080BEABAAAAAA3E000009
:1000B0000000BF000000803F000000000008417801
:1000C000D3BB4387D1133D190E3CC3BD4282AD2B38
:1000D0003E68EC8276BED98FE1A93E4C80EFFFBE30
:1000E00001C4FF7F3F00000000000000000024006A
:1000F00027002A0000000000250028002B00000037
:10010000000023002600290004040404040404045D
:1001100002020202020203030303030301020408B2
:100120001020408001020408102001020408102061
:1001300000000008000201000003040700000000A6
:1001400000000000E90511241FBECFEFD8E0DEBF9C
:10015000CDBF11E0A0E0B1E0E0E3F3E102C0059023
:100160000D92A234B107D9F721E0A2E4B1E001C0B9
:100170001D92AC36B207E1F710E0C3EAD0E004C04C
:100180002197FE010E949009C23AD107C9F70E9447
:10019000FE020C9496090C940000833081F028F440
:1001A000813099F08230A9F008958730A9F0883025
:1001B000C9F08430B1F4809180008F7D03C08091BC
:1001C00080008F7780938000089584B58F7784BDF9
:1001D000089584B58F7DFBCF8091B0008F77809399
:1001E000B00008958091B0008F7DF9CFCF93DF9359
:1001F000282F30E0F901E05DFE4F8491F901E45EC3
:10020000FE4FD491F901E85FFE4FC491CC23A1F0D9
:1002100081110E94CD00EC2FF0E0EE0FFF1FE250A5
:10022000FF4FA591B491EC91ED2381E090E009F4AA
:1002300080E0DF91CF91089580E090E0FACF1F93A6
:10024000CF93DF93282F30E0F901E05DFE4F8491DA
:10025000F901E45EFE4FD491F901E85FFE4FC491CD
:10026000CC23A9F0162F81110E94CD00EC2FF0E0D5
:10027000EE0FFF1FEC50FF4FA591B4918FB7F8948C
:10028000EC91111108C0D095DE23DC938FBFDF9174
:10029000CF911F910895DE2BF8CFCF93DF9390E09D
:1002A000FC01E45EFE4F2491885F9E4FFC01849127
:1002B0008823C9F090E0880F991FFC01E651FF4F99
:1002C000A591B491FC01EC50FF4FC591D4916111FF
:1002D0000DC09FB7F8948C91209582238C938881D0
:1002E000282328839FBFDF91CF910895623051F476
:1002F0009FB7F8943C91822F809583238C93E8815B
:100300002E2BEFCF8FB7F894EC912E2B2C938FBF21
:10031000EACF1F93CF93DF93182FEB0161E00E9488
:100320004D01209739F460E0812FDF91CF911F912B
:100330000C941F01CF3FD10511F461E0F5CFE12FFF
:10034000F0E0E05DFE4FE491E33031F140F4E13064
:10035000B1F0E230E1F0C038D1057CF7E4CFE7300E
:1003600029F1E83059F1E430B1F7809180008062E2
:1003700080938000D0938B00C0938A0004C084B522
:10038000806884BDC7BDDF91CF911F91089584B56A
:10039000806284BDC8BDF7CF809180008068809363
:1003A0008000D0938900C0938800EDCF8091B00089
:1003B00080688093B000C093B300E5CF8091B00017
:1003C00080628093B000C093B400DDCF8E50806413
:1003D00080937C0080917A00806480937A00809181
:1003E0007A0086FDFCCF8091780090917900089585
:1003F0008091590190915A01029739F520E030E03F
:1004000040E450EC60915B0170915C0180915D0172
:1004100090915E010E94ED080E94E10660935F01E9
:1004200070936001809361019093620181E090E09C
:1004300090935A018093590110925B0110925C01D4
:1004400010925D0110925E01089560E070E0CB01B2
:10045000E5CF4F925F926F927F928F929F92AF9271
:10046000BF92CF92DF92EF92FF92CF93DF936B0117
:100470007C0120E030E0A9010E94620687FD69C08E
:1004800020E030E040E85FE3C701B6010E942208A7
:1004900018160CF462C020E030E040E052E4C701DE
:1004A000B6010E94ED084B015C010E941307EB01AD
:1004B0006032710514F0CFE1D0E0FE01EE0FFF1FB6
:1004C000E050FF4F6081718190E080E00E94490719
:1004D0000E9471086B017C01FE01EE0FFF1FEE5FB1
:1004E000FE4F6081718190E080E00E9449070E9488
:1004F00071082B013C01BE01DD0F880B990B0E9496
:100500004B079B01AC01C501B4010E94F5054B01ED
:100510005C01A7019601C301B2010E94F5059B0190
:10052000AC01C501B4010E94ED08A70196010E942B
:10053000F605DF91CF91FF90EF90DF90CF90BF90C5
:10054000AF909F908F907F906F905F904F900C94A2
:10055000E106C12CD12C76019ECFC12CD12C20E8F4
:10056000E22E2FE3F22E97CF1F920F920FB60F922B
:1005700011242F933F938F939F93AF93BF938091B9
:10058000550190915601A0915701B09158013091B9
:10059000540123E0230F2D3758F50196A11DB11DFD
:1005A000209354018093550190935601A0935701D5
:1005B000B09358018091500190915101A091520146
:1005C000B09153010196A11DB11D809350019093EC
:1005D0005101A0935201B0935301BF91AF919F91EC
:1005E0008F913F912F910F900FBE0F901F901895F4
:1005F00026E8230F0296A11DB11DD2CFCF93DF9322
:10060000CDB7DEB728970FB6F894DEBF0FBECDBFCB
:10061000789484B5826084BD84B5816084BD85B5DD
:10062000826085BD85B5816085BD80916E008160E9
:1006300080936E001092810080918100826080938F
:100640008100809181008160809381008091800091
:100650008160809380008091B10084608093B100BC
:100660008091B00081608093B00080917A008460B6
:1006700080937A0080917A00826080937A008091E2
:100680007A00816080937A0080917A0080688093FC
:100690007A001092C10062E084E00E944D0160E0A7
:1006A00081E10E944D0161E083E00E944D0161E023
:1006B00089E00E944D0161E08AE00E944D0161E005
:1006C0008BE00E944D0183E28093B00081E0809333
:1006D000B10082E88093800089E1809381008FEFF0
:1006E00090E090938700809386000FEF10E052E037
:1006F000252E312C8FB7F894209155013091560159
:10070000409157015091580129833A834B835C8370
:100710008FBF20934C0130934D0140934E01509375
:100720004F018EE00E94E6016C018FE00E94E6011D
:100730007C0180E10E94E601BC01990F880B990BB6
:100740000E944B0720E030EC4FE754E40E9467061C
:100750002B013C01B601DD0C880B990B0E944B0765
:1007600020E030EC4FE754E40E9467060E94290223
:100770004B015C01B701FF0C880B990B0E944B07E2
:1007800020E030EC4FE754E40E9467060E94290203
:100790006B017C0120E030E040E85FE3C501B4017B
:1007A0000E94620687FD1CC120E030E040E854E46E
:1007B000C501B4010E94220818160CF418C120E0EB
:1007C00030E040E85FE3C701B6010E94620687FDA2
:1007D00015C120E030E040E854E4C701B6010E94B2
:1007E000220818160CF411C120E030E0A901C30161
:1007F000B2010E94620687FD0FC120E030E040E8B0
:100800005FE3C301B2010E94220818160CF408C16C
:1008100084E00E94F60020914901211103C091E07B
:10082000813009F090E090934A01213011F491E079
:10083000811190E090934B018093490191110E94A6
:10084000F80181E10E94F60020914601211103C0C8
:1008500091E0813009F090E090934701213009F454
:10086000811120E0209348018093460191110E945C
:10087000F8018091420190914301A0914401B0910F
:10088000450129813A814B815C8182179307A40736
:10089000B50709F496C12093420130934301409378
:1008A0004401509345018091590190915A0101975B
:1008B00021F520E030E048EC51E4C501B4010E948C
:1008C000ED0820E030E040E85AE30E94ED084B01DB
:1008D0005C0120E03AE647EC51E40E94220887FDE3
:1008E000A6C030925A012092590110925B011092D9
:1008F0005C0110925D0110925E018091590190910E
:100900005A01029709F0F3C080905B0190905C015E
:10091000A0905D01B0905E0120E030E040E450EC3A
:10092000C501B4010E94ED080E94E1069B01AC01E3
:10093000C301B2010E94ED086093630170936401EA
:10094000809365019093660120E030E048EC51E42B
:10095000C701B6010E94ED0820E030E040E85AE30C
:100960000E94ED082FE632E143E85AE30E94ED08C9
:10097000A50194010E94F60560935B0170935C01F0
:1009800080935D0190935E0120E030E040E85FE3FA
:100990000E94220887FDB9C010925A011092590195
:1009A00010925B0110925C0110925D0110925E0149
:1009B0001092630110926401109265011092660119
:1009C00091E0909367012AE037ED43E25CE32093E6
:1009D00068013093690140936A0150936B0187C0AD
:1009E000812C912C40E8A42E4FE3B42EE8CE812C2C
:1009F000912C30E8A32E34E4B32EE1CEC12CD12CBF
:100A000020E8E22E2FE3F22EEFCEC12CD12C90E87D
:100A1000E92E94E4F92EE8CE412C512C3201F8CE87
:100A2000412C512C80E8682E8FE3782EF1CE8091F6
:100A30005B0190915C01A0915D01B0915E018983A1
:100A40009A83AB83BC8320E030E040E450ECBC01EF
:100A5000CD010E94ED080E94E1066D837E838F83A5
:100A6000988720915F013091600140916101509120
:100A7000620160E070E080E89FE30E94F5052D814F
:100A80003E814F8158850E94ED089B01AC0160E0DA
:100A900070E080E89FE30E94F505A30192010E94A7
:100AA000ED086093630170936401809365019093F6
:100AB00066012FE632E143E85AE3C501B4010E9422
:100AC000ED0829813A814B815C810E94F605609393
:100AD0005B0170935C0180935D0190935E0120E067
:100AE00030E040E85FE30E94220887FFFACE809161
:100AF000590190915A01892B41F41092630110928F
:100B0000640110926501109266018091670188234B
:100B100039F12FE632E143E85AE3609168017091C0
:100B2000690180916A0190916B010E94F5056093C3
:100B300068017093690180936A0190936B0120E0D2
:100B400030E0A9010E946206181654F01092670165
:100B5000109268011092690110926A0110926B0163
:100B600020E030E04FE753E460916301709164014D
:100B700080916501909166010E94ED0820E030E0CF
:100B800040E05FE30E94F6050E9413076B018BE0D3
:100B90000E94890130EA3C9DC0013D9D900D1124C9
:100BA000B8010E94680983E00E948901B8016C19AC
:100BB0007D098AE00E9489016091670189E00E94B5
:100BC0001F0140E050E0452B09F494CD0E94000045
:100BD00091CDE9E4F1E081E0808311821282E6E4C4
:100BE000F1E010821182128208955058BB27AA2783
:100BF0000E940D060C94E8070E94DA0738F00E9464
:100C0000E10720F039F49F3F19F426F40C94B00763
:100C10000EF4E095E7FB0C94AA07E92F0E94F90770
:100C200058F3BA17620773078407950720F079F421
:100C3000A6F50C941B080EF4E0950B2EBA2FA02DF0
:100C40000B01B90190010C01CA01A0011124FF2779
:100C5000591B99F0593F50F4503E68F11A16F04074
:100C6000A22F232F342F4427585FF3CF4695379573
:100C70002795A795F0405395C9F77EF41F16BA0B38
:100C8000620B730B840BBAF09150A1F0FF0FBB1FE6
:100C9000661F771F881FC2F70EC0BA0F621F731F2F
:100CA000841F48F4879577956795B795F7959E3F8C
:100CB00008F0B0CF9395880F08F09927EE0F97951D
:100CC000879508950E94860708F481E008950E94A0
:100CD0007B060C94E8070E94E10758F00E94DA07AF
:100CE00040F029F45F3F29F00C94AA0751110C94AD
:100CF0001C080C94B0070E94F90768F39923B1F31C
:100D0000552391F3951B550BBB27AA276217730731
:100D1000840738F09F5F5F4F220F331F441FAA1FC5
:100D2000A9F335D00E2E3AF0E0E832D09150504081
:100D3000E695001CCAF72BD0FE2F29D0660F771F2F
:100D4000881FBB1F261737074807AB07B0E809F015
:100D5000BB0B802DBF01FF2793585F4F3AF09E3F9A
:100D6000510578F00C94AA070C941C085F3FE4F33B
:100D7000983ED4F3869577956795B795F7959F5FDD
:100D8000C9F7880F911D9695879597F90895E1E029
:100D9000660F771F881FBB1F621773078407BA0788
:100DA00020F0621B730B840BBA0BEE1F88F7E095E3
:100DB000089529F416F00C94AA070C941B080C94BF
:100DC000B0070E940108A8F39638A0F707F80F9221
:100DD000E8942BE33AEA48EB5FE70E9403090F929D
:100DE0000F920F924DB75EB70F920E94B908E8E6D6
:100DF000F0E00E94B3074F915F91EF91FF91E5956D
:100E0000EE1FFF1F49F0FE57E0684427EE0F441F16
:100E1000FA95E1F74195550B0E9433080F9007FEB4
:100E20000C94270808950E941A076894B1110C9435
:100E30001C0808950E94010888F09F5798F0B92F68
:100E40009927B751B0F0E1F0660F771F881F991FFF
:100E50001AF0BA95C9F714C0B13091F00E941B087E
:100E6000B1E008950C941B08672F782F8827B85F8E
:100E700039F0B93FCCF3869577956795B395D9F757
:100E80003EF490958095709561957F4F8F4F9F4F61
:100E90000895E89409C097FB3EF49095809570956D
:100EA00061957F4F8F4F9F4F9923A9F0F92F96E9B6
:100EB000BB279395F695879577956795B795F1112B
:100EC000F8CFFAF4BB0F11F460FF1BC06F5F7F4FC8
:100ED0008F4F9F4F16C0882311F096E911C07723DA
:100EE00021F09EE8872F762F05C0662371F096E8E3
:100EF000862F70E060E02AF09A95660F771F881FB2
:100F0000DAF7880F9695879597F90895990F000855
:100F1000550FAA0BE0E8FEEF16161706E807F907CB
:100F2000C0F012161306E407F50798F0621B730B66
:100F3000840B950B39F40A2661F0232B242B252BE7
:100F400021F408950A2609F4A140A6958FEF811D8A
:100F5000811D089597F99F6780E870E060E008952B
:100F60009FEF80EC0895DF93CF931F930F93FF9231
:100F7000EF92DF927B018C01689406C0DA2EEF01BC
:100F80000E940009FE01E894A591259135914591B3
:100F90005591A6F3EF010E940D06FE019701A801ED
:100FA000DA9469F7DF90EF90FF900F911F91CF9146
:100FB000DF91089500240A941616170618060906EC
:100FC000089500240A9412161306140605060895BF
:100FD000092E0394000C11F4882352F0BB0F40F447
:100FE000BF2B11F460FF04C06F5F7F4F8F4F9F4F87
:100FF000089557FD9058440F551F59F05F3F71F009
:101000004795880F97FB991F61F09F3F79F087956F
:101010000895121613061406551FF2CF4695F1DFF8
:1010200008C0161617061806991FF1CF8695710588
:10103000610508940895E894BB2766277727CB01BC
:1010400097F908950E94860708F48FEF08959B0191
:10105000AC0160E070E080E89FE30C9467060C94BC
:10106000AA070C945A090E940108D8F39923C9F3DE
:10107000940F511DA3F39150504094F059F08823E0
:1010800032F0660F771F881F91505040C1F79E3F86
:1010900051052CF7880F911D9695879597F908951E
:1010A0005F3FACF0983E9CF0BB278695779567959F
:1010B000B79508F4B1609395C1F7BB0F58F711F4D9
:1010C00060FFE8CF6F5F7F4F8F4F9F4FE3CF0C9450
:1010D0001C0816F00C945A090C94B00768940C94F0
:1010E000AA070E940108A8F39923C1F3AEF3DF9386
:1010F000CF931F930F93FF92C92FDD2788232AF0E8
:101100002197660F771F881FDAF720E030E040E86C
:101110005FEB9FE3883920F0803E38F021968F778F
:101120000E94F605E0E9F0E004C00E94F605EDEB50
:10113000F0E00E94B3078B01BE01EC01FB2E6F575C
:1011400071097595771F880B990B0E944B0728E151
:1011500032E741E35FE30E940009AF2D9801AE0141
:10116000FF900F911F91CF91DF910E940D060C947B
:10117000E807FA01DC01AA0FBB1F9B01AC01BF57B6
:1011800028F4222733274427507820C0B75190F401
:10119000AB2F0024469537952795011CA395D2F3D4
:1011A000002071F0220F331F441FB395DAF30ED0E5
:1011B0000C94F50561307105A0E88A07B94630F452
:1011C0009B01AC016627772788279078309621F01D
:1011D000208331834283538308950E9400090C9435
:1011E000E8070E94DA0738F00E94E10720F0952313
:1011F00011F00C94AA070C94B00711240C941C084D
:101200000E94F90770F3959FC1F3950F50E0551FA9
:10121000629FF001729FBB27F00DB11D639FAA274B
:10122000F00DB11DAA1F649F6627B00DA11D661F9A
:10123000829F2227B00DA11D621F739FB00DA11DBB
:10124000621F839FA00D611D221F749F3327A00D75
:10125000611D231F849F600D211D822F762F6A2F11
:1012600011249F5750409AF0F1F088234AF0EE0F76
:10127000FF1FBB1F661F771F881F91505040A9F7A3
:101280009E3F510580F00C94AA070C941C085F3F08
:10129000E4F3983ED4F3869577956795B795F795DF
:1012A000E7959F5FC1F7FE2B880F911D9695879557
:1012B00097F908959F3F31F0915020F487957795E5
:1012C0006795B795880F911D9695879597F908951D
:1012D00097FB072E16F4009407D077FD09D00E94E3
:1012E0007C0907FC05D03EF4909581959F4F0895A9
:1012F000709561957F4F0895AA1BBB1B51E107C0F4
:10130000AA1FBB1FA617B70710F0A61BB70B881F95
:10131000991F5A95A9F780959095BC01CD01089524
:10132000EE0FFF1F0590F491E02D0994F894FFCF84
:1013300000046B03EC027F022102D2018D015301F4
:101340002101F600D200B300980081006E005D001C
:101350004F00430038002F00280021001B00170019
:1013600012000F000C000900070005000400020035
:0213700001007A
:00000001FF
